:03000000020008F3
:0300610002000397
:050003001200C680FEA2
:09006400AA82AB83EA4BB401004F
:0B006D00E433FCE4BA0104BB00010412
:070078004C6004900001221E
:0E007F00EA24FFF582EB34FFF583C002C003D4
:08008D001200648582088583DE
:0C00950009D003D0028A828B830200E5B0
:0D00A100439840438920758DFD43878022E0
:0800AE00AA82AB83C2998A9972
:0400B6003099FD225E
:0C00BA003098FDAA997B008A828B83227B
:0D00C6001200A190000A1200AE900014126A
:0900D30000AE900003120064125B
:0900DC0000AE1200BA90000522EA
:06003700E478FFF6D8FD9D
:080015007900E94400601B7A48
:05001D000090010678CF
:030022000075A0C6
:0A00250000E493F2A308B8000205FE
:08002F00A0D9F4DAF275A0FF7C
:0B00E500E5828508F0A4C582C0F0850C
:0A00F00009F0A4D0F025F0C58385C7
:0800FA0008F0A42583F5832220
:08003D007800E84400600A7934
:030045000075A0A3
:0600480000E4F309D8FCFE
:08004E007800E84400600C7921
:0B00560000900000E4F0A3D8FCD9FAF1
:03000800758109F6
:0A000B00120102E582600302000307
:0401020075820022E0
:00000001FF
